:1000000000308A009C2D00000A108A100A11820715
:100010003E347F34713459344D347F343E3440346F
:1000200042347F347F34403440340034623473349B
:10003000593449346F3466340034223463344934DB
:1000400049347F343634003418341C341634533475
:100050007F347F34503427346734453445347D341D
:10006000393400343C347E344B34493479343034C0
:10007000003403340334713479340F3407340034DA
:1000800036347F34493449347F34363400340634CE
:100090004F34493469343F341E3400341C343E3408
:1000A00063344134413463342234083408343E34F8
:1000B0003E34083408340034083408340834083432
:1000C00008340834003400340034603460340034C0
:1000D0000034003400340034063409340934063462
:1000E0000034003400340034003400340034003470
:1000F0000A108A100A11820700348034C034E034B8
:10010000F034F834FC34FE34FF34FF348316010835
:10011000C73908388100831290010730990083168F
:10012000050803308312A000A00B942819088C1135
:10013000831699010C3085008312C42D7D30840014
:1001400000080319B1280130A100A001A00BA628C6
:10015000A10BA5284A30A000A00BAC28AF28800B2B
:10016000A328003408308316A000A0080319D12862
:100170008512831285127F088039031DC4288316D7
:10018000051283120512C82883160512831205165C
:1001900083168512831285160310FF0D8316A003A4
:1001A000B5288312003483160510831205107E08CB
:1001B000FF00B22000347C0807394038FD00FE0003
:1001C000D3207B087F398038FD00FE00D320003427
:1001D00083160510831205147B08FF00B22000343B
:1001E000831605108312051483168510831285105B
:1001F0006430FD009E208316851083128514213003
:10020000FE00D320C830FE00D3201330FE00D320E0
:100210002030FE00D3200930FE00D320FB01FC017A
:10022000DB200130F500F830F400F408031D1B2931
:10023000F50803192229FB01E82074080319F503C6
:10024000F40315290830FE00D3200C30FE00D32023
:10025000FB01FC01DB20C52D7508FB007608FC00C6
:10026000DB207708F9007808770779020318452919
:10027000790883169B009C131C141A08FA007A084C
:10028000FB008312E820F90A332900344030F500DE
:10029000F601F7011330F8002C214030F500013051
:1002A000F6001330F700F8002C214030F500023042
:1002B000F6002630F7001330F8002C214A30F50004
:1002C0000330F6003930F7000930F8002C214830AF
:1002D000F5000430F6004230F7000930F8002C2118
:1002E0000230F5000530F6004B30F7005030F800D2
:1002F0002C21FB010130FC00DB20FF30FB00E8205B
:10030000F4017408383C031C8A290130FB00E82002
:10031000F40A81294330FB00E820FF30FB00E8208D
:10032000FB010230FC00DB20FF30FB00E8203A300C
:10033000FB000230FC00DB200830FB00E820FF302F
:10034000FB00E820FB010330FC00DB20FF30FB005A
:10035000E820F40174081B3C031CB529FB01E820CC
:100360002030FB00E820F40AAA29FB01E820213014
:10037000FB00E820FF30FB00E820FB01E8203030E4
:10038000FB00E8204830FB00E8204830FB00E82074
:100390003030FB00E820FB010430FC00DB203F3064
:1003A000FB00E820F4017408383C031CDC292030F1
:1003B000FB00E820F40AD3292430FB00E8203F307A
:1003C000FB00E820E62D8316051183120511A630E7
:1003D000A000A00BE929000083160515A6308312A2
:1003E000A000A00BF129000083160515831200342C
:1003F000FE017E08073C031C172A83160511831291
:100400000511022A0310FD0C0318082A0511092AF8
:1004100005158316051113308312A000A00B0E2AB8
:10042000112A83160515142AFE0A8312F9290034AD
:10043000FD017D08073C031C3A2A8316051183122F
:100440000511222A8316051502308312A000A00B85
:10045000272A00008316051583120519312A031077
:10046000322A0314FE0C2730A000A00B352A382AAC
:10047000FD0A192A7E08A1000034A001A101760816
:1004800003107718A007A00CA10CF718A007A00C68
:10049000A10C7719A007A00CA10CF719A007A00CBC
:1004A000A10C771AA007A00CA10CF71AA007A00CAA
:1004B000A10C771BA007A00CA10CF71BA007A00C98
:1004C000A10C0034F5017508063C031C742A74085D
:1004D000F6000730F7003D22750821070420F800D8
:1004E000FB00E820F50A632A0034A101A201A00163
:1004F000A3017708031D7F2A76080319992A103073
:10050000F8000310F40DF50DA00DA30D77082302DC
:10051000031D8C2A76082002031C952A7608A00267
:10052000031CA3037708A3020314A10DA20DF80B6B
:10053000812A0034F401E321CC30FD00F82144305D
:10054000FD00F821F408031DA92A18222108F4004F
:10055000A22AE321CC30FD00F821BE30FD00F821B5
:1005600018222108F50018222108F6007608F80064
:100570007508F7007808FE007708FD008E30A000AF
:100580007E08A1007D08A200A301FE1FCC2AA109BC
:10059000A209A20A0319A10AA108031DD92A220847
:1005A000A100A2010830A002A108031DD92AA001C0
:1005B000E22A0310A11BE02AA20DA10DA003D92A53
:1005C000FE1FA1132308FC002208FB002108FA00EB
:1005D0002008F900C830FD009E207908A0007A08A4
:1005E000A1007B08A2007C08A3002308F7002208D2
:1005F000F6002108F5002008F4008E30A0007408F1
:10060000A0027508A2007608A100A217A00803198D
:10061000142B0310A208031D102BA1080319142B7F
:10062000A20CA10CA00B092BF51F1B2BA109A209E1
:10063000A10A0319A20A2208AC002108AB00AA01F2
:100640000430FB000330FC00DB202C08003C031CC2
:10065000302BAC012B1C2E2B0130AA00B001452BF6
:100660000C30F4006222AC012B08003CAB002C08DB
:10067000031C2C0F3D2B01303E2B013CAC002B1CEE
:10068000432B0130AA000130B0000310AC0CAB0CBE
:100690002B08F0002C08F5002B08F400F70164305B
:1006A000F60075222108AD002D08F6006430F70031
:1006B0003D222108AB020030031C0130AC022C08A3
:1006C000F5002B08F400F7010A30F6007522210826
:1006D000AE002E08F6000A30F7003D222108AB02DA
:1006E0000030031C0130AC022B08AF00AD08031D25
:1006F000802B0F30AD00AE08031D802B0F30AE00F5
:02070000F32DD7
:100800004C30FB00FC01DB200430FB00E8204C30C6
:10081000FB000130FC00DB20FB01E8204C30FB003A
:100820000230FC00DB20FB01E8204C30FB000330F1
:10083000FC00DB20FB01E8202E080F3C031D2B2CC5
:100840004C30FB000330FC00DB202F087820F40044
:10085000FB00E820AC2C2E0B402C4C30FB0003306E
:10086000FC00DB20FF30FB00E8204C30FB000230B6
:10087000FC00DB202F087820F400FB00E820AC2CE3
:100880002E08023C031D5F2C4C30FB000330FC00A3
:10089000DB20FF30FB00E8204C30FB000230FC0086
:1008A000DB20FF30FB00E8204C30FB000130FC0077
:1008B000DB202F087820F400FB00E820AC2C2E0869
:1008C000033C031D8D2C4C30FB000330FC00DB206F
:1008D000FF30FB00E8204C30FB000230FC00DB2046
:1008E000FF30FB00E8204C30FB000130FC00DB2037
:1008F000FF30FB00E8204C30FB00FC01DB202F0820
:10090000053C031C892C2F087820F400FB00E8200C
:100910008C2CF830FB00E820AC2C4C30FB00033072
:10092000FC00DB20FF30FB00E8204C30FB000230F5
:10093000FC00DB20FF30FB00E8204C30FB000130E6
:10094000FC00DB20FF30FB00E8204C30FB00FC010A
:10095000DB20F830FB00E820572EF4017408383C07
:10096000031CC12C35307407F90001307407353E83
:1009700084000008FB00790884007B088000F40AEA
:10098000AE2CB008031DCE2C70082A3C031CCB2CC7
:100990007008EE00CD2C2A30EE00DA2C300BDA2C69
:1009A00070080E3C031CD82C70088038EE00DA2C3E
:1009B0008E30EE00F4017408383C031C9B2D35305A
:1009C000740784000008F50075087F3C031C082D9F
:1009D0000310750CF800A0307807F9002130FA00F8
:1009E0000318FA0A790883169B009C131C141A0832
:1009F000F700B6307807F9002130FA000318FA0A38
:100A000079089B009C131C141A08F600282D8312E9
:100A10008030F5020310750CF800D0307807F9002B
:100A20002130FA000318FA0A790883169B009C13F8
:100A30001C141A08F700D7307807F9002130FA00A3
:100A40000318FA0A79089B009C131C141A08F60074
:100A5000770F2B2D982D760B3A2D01307407F90066
:100A6000FB007608FC008312DB207708FB00E820FF
:100A7000452D831601307407F900FB000130FC009E
:100A80008312DB200130FB00E8207608023C031DC6
:100A9000542D01307407F900FB007608FC00DB20C0
:100AA0007708FB00E8205D2D01307407F900FB009A
:100AB0000230FC00DB20FB01E8207608033C031D2C
:100AC0006F2D741C642DF71601307407F900FB00BC
:100AD0007608FC00DB207708FB00E8207E2D013043
:100AE0007407F900FB000330FC00DB20741C7C2D34
:100AF0002030FB00E8207E2DFB01E8207608043C36
:100B0000031D8D2D01307407F900FB007608FC00F1
:100B1000DB207708FB00E820972D01307407F900EF
:100B2000FB000430FC00DB202030FB00E8208316B3
:100B3000F40A8312DB2C5C2E03081F3983005F301C
:100B4000A0002130840083138001840AA00BA42D0F
:100B50002030A000A030840083138001840AA00B01
:100B6000AD2DA00184011F308305613083168F00F5
:100B700083121F1383161F109F101F119F11073020
:100B800083129900A5018628F028FE3083169B0069
:100B90009C131C141A088312B300FF3083169B00A9
:100BA0009C131C141A088312B4003308B2003408D2
:100BB000B100F1017108393C031CE52D3530710796
:100BC0008400FF308000F10ADA2D4629F301F2019A
:100BD00073083202031C5B2E031DF22D31087202D2
:100BE00003185B2E9A2AB008031D182E3D30FB0017
:100BF000FC01DB20FB01E820FB01E8203D30FB008D
:100C00000130FC00DB20FB01E820FB01E8203D3047
:100C1000FB000230FC00DB20FB01E820FB01E820A8
:100C20000130FB00FC01DB202D08F40062223F2E86
:100C30003D30FB00FC01DB200830FB00E8200830E1
:100C4000FB00E8203D30FB000130FC00DB200830D9
:100C5000FB00E8200830FB00E8203D30FB000230BC
:100C6000FC00DB200830FB00E8200830FB00E82017
:100C70000130FB00FC01DB200C30F40062222E0866
:100C8000F40062222F08F40062220D30F400622288
:100C90002A0B4E2E0530F4006222502EF4016222FF
:100CA0000E30F40062220A30F4006222002CF20AB4
:0C0CB0000319F30AE82DAD2CE62D6300BB
:0207FE00803445
:104200009400A200AA00940080009C00A200A200DA
:104210009C000000F800040004000400F800000006
:10422000000080008000A400B200AA00A40080006A
:104230009C00A200A2009C000000FF000000000003
:104240000000FF0000000800800080008000800067
:104250008400BE0080009C00A200A2009C00000020
:10426000FF00000000000000FF00000008008000C8
:104270008000FF00800080008000FF000000080038
:10428000800080000E001F003F003F002F002F0025
:1042900031001F000E00FE00120012003200CC00A0
:1042A0000000C800A800A800F80000000000FE0000
:1042B0008200820082007C000000FA000000000002
:1042C000FE001000280044008200C800A800A800DA
:1042D000F8000000FE0000000000FE0082008200E6
:1042E00082007C0000007000A800A800B000000060
:1042F00000004C009200920064000000FA000000F0
:1043000000007C0082008200920074000000000027
:1043100080000000700088008800500000007000DD
:104320008800880070000000F80008000800F8000D
:0643300008000800F00087
:10434000200010000800040002000100800040006E
:10435000200010000800040002000100810041005C
:104360002100110009000500030002000300030002
:104370000300030003000300020002000200020029
:104380000200020002000200010001000100010021
:08439000010001000100010021
:1043A000400080002100220024002800300003008B
:0C43B000030004000400040004000400EA
:0443FC0000000500B8
:02400E00D430AC
:00000001FF
